:030000000219FDE5
:03000B000200AA46
:03002B0002018748
:03005B0002034459
:0300730002033154
:1000800002030406080C10182030406080040608A3
:100090000C10182030406080A0C00003070F1F0D17
:1000A0000D04050D050305030302C2AF306308C24A
:1000B0006385798AD2AF32C0D0C0E0206221E525C5
:1000C0006016E473E525F4C3334009758A00D263F2
:1000D000F57901D6F58AD262D0E0D0D0D2AF32C362
:1000E000E526334009758A00D263F57901F0F58A77
:1000F000C262E526F4602F30682520720DD0E0D072
:10010000D0C292C294C296D2AF32C292C294C29668
:10011000206F0C206609740AD5E0FDE57B4290D083
:10012000E0D0D0D2AF32758A00D263757900C28D2B
:10013000D262211F01C4306805206602D29201C438
:10014000306805206602D29401C43068052066023A
:10015000D29601C4C29330680A2066077408D5E0BD
:10016000FDD29201C4C29530680A2066077408D592
:10017000E0FDD29401C4C29730680A206607740873
:10018000D5E0FDD29601C4C2AFC2AD53E6EFC0D0F8
:10019000C0E0D2D3D2AFE57A6009E5776005757724
:1001A0000041DE757701C2CEE52A6007207449154B
:1001B0002A21F87800790020742EE580307E01F441
:1001C00030E60278FF53DACF207E0343DA20307E18
:1001D0000343DA10C2D8C271E580307E01F430E604
:1001E0000279FFC3E89970CB306103752A18207437
:1001F00003752A18885CD27020740DE52B600415F5
:100200002B410843DA01C2D82070024177A85C2054
:100210006102C2702074367982B70431C3E894F069
:10022000400374F0F8E8C4540F28F87984B7030247
:10023000414DC313C3138721200802C313200A06AC
:10024000C3C898F8414D28F8500374FFF88822E598
:100250002D54066022206B1FE536C333C333F8E507
:1002600064C313C313F9C3952240028922E82522EF
:10027000F52250037522FF7882B60459852224A8FE
:1002800024C3E52495614002A861C3E89563400258
:10029000A8638825E566700241C8C3E8AA669A503B
:1002A00003E8FAE4F9EAC333FBE568F45B29400D9F
:1002B0002567F8E56760021567400B41C80AC3E58A
:1002C000679A5002056778FF8826C26FC3E52694B7
:1002D000F84002D26FC3E52594404002D26420CF9B
:1002E0000AD0E0D0D043E610D2AD32C2CF053AE515
:1002F0007A6009E57860057578006127757801787E
:1003000001E52A6005307402152AC3E55C940140BA
:1003100005755F006127756000756900E55F240160
:10032000F55F5003755FFFD0E0D0D043E610D2AD4B
:1003300032C2AF53E67F7592FA7593FFC260759132
:1003400004D2AF32C2AF53E6EFC2ADC0D0C0E0C0FE
:10035000F0D2D3D2AFA8FBA9FCE57A6007C3E913BA
:10036000F9E813F8C2D830710261B653DACF207EB3
:100370000343DA10307E0343DA20D271E580307E09
:1003800001F420E602618D88278928A1E353DACFA2
:10039000207E0343DA20307E0343DA10C2D8C271D4
:1003A000307402A1CF7800E580307E01F430E6029F
:1003B000A1CF885CA1B753DACF207E0343DA203087
:1003C0007E0343DA10C271206102818F53DACF209D
:1003D0007E0343DA10307E0343DA20C2D8D271881C
:1003E000578958C3E89555F8E99556F97B007E087A
:1003F0007A00C3E8948CE994005005755B00818114
:10040000882178A2E6A8216055C3E894C8E9940041
:100410005008E4D2E4FB7A0A815CC3E89468E9946A
:10042000015008E4D2E3FB7A0F815CC3E894D0E981
:1004300094025008E4D2E2FB7A1E815CC3E894A0E7
:10044000E994055008E4D2E1FB7A3C815CC3E8946E
:1004500098E994085008E4D2E0FB7A787E00C3E87B
:100460009559FCE9955AFD30E70AECF42401FCEDBE
:0E047000F43400FD755B00C3EC9AED9E500362
:10047E00755B018859895A8557558558567802A15A
:10048E00B7C3E89527F8E99528F9307C02A19B308F
:10049E007B02A19B307A02A19420750281B2E9FD04
:1004AE00E8FC81D1E9C313F9E813F8307902A1947D
:1004BE00E9C313F9E813F8307802A194E9C313FDE8
:1004CE00E813FC20612CC3EC941CED9402400281D5
:1004DE00E8ED701EC3EC94C850180529E52970028A
:1004EE001529C3E529940A5002A1CF755C00D2707C
:1004FE00A1CFE529600215297888E6F97400207FDE
:10050E00087896B90302789EE624FAFEE43400FFDA
:10051E00C3EC9EFCED9FFD9208B90310A208500794
:10052E00207609D276A13A307602C276A20850160B
:10053E00B9030DECF42401FCEDF43400FD02055476
:10054E0078007900A19BB90315EC33FCED33FDC3A4
:10055E00EC940AFCED9400FD50047C007D00C3EC8D
:10056E0094FFED9400400678FF7900A19BEC857214
:10057E00F0A4C5F0A2F733F8790040030205B7786E
:10058E00FF79000205B7E9C313F9E813F8307C0EC2
:10059E00E9600278FFC3E81338F8E43400F9C3E8E1
:1005AE0094FFE99400400278FF885CD270206102CB
:1005BE00A1CF741FF4552F4BF52FC274EB7002D2DE
:1005CE0074752A18307403752A0A306102A1E3206B
:1005DE00740353DAFE207403752B06D0F0D0E0D0EE
:1005EE00D0D2AD43E610327901020613790302062A
:1005FE0013790A020613791E020613796402061392
:10060E0079C80206137817E4D5E0FDD8FAD9F62298
:10061E007A147B7802063A7A107B8C02063A7A0DAF
:10062E007BB402063A7A0B7BC802063A7902E4C220
:10063E0095D5E0FDD294D5E0FDC294D5E0FDD295DE
:10064E00D5E0FDE920E002D29230E002D296E573C9
:10065E00D5E0FDE920E002C29230E002C296749627
:10066E00D5E0FDD9C9EAF8D5E0FDD8FBDBBEC295D1
:10067E0022C37C007D0075F00005F0EA33FAEB33FF
:10068E00FB50F6EB13FBEA13FAC3E9FFE8FEE89A18
:10069E00F8E99BF95004EFF9EEF8B3EC33FCED33C7
:1006AE00FDD5F0DFEDF9ECF822E889F08A20D2D4FE
:1006BE00F8A9F07B0030F70B7BFFF42401F8E9F486
:1006CE003400F9E88520F0A4ADF0F8E98520F0A417
:1006DE00AFF0FEED2EF974003FFA7C04C3EA13FA74
:1006EE00E913F9E813F8DCF48BF030F70AE8F42498
:1006FE0001F8E9F43400F9E889F0C2D4F8A9F0223F
:10070E007882B60403020769C3E55C9401400302D4
:10071E000733852224E4F544F545F546F547F548BB
:10072E00C26E0207697882E6FCD26EE522F5237866
:10073E003879C7AA40AB41C3EB13FBEA13FAEC14AA
:10074E006013C3EB13FBEA13FAEC14146007C3EB4C
:10075E0013FBEA13FAD17F8844894522C3E54495F9
:10076E0023F8E5459400F9500CC3E89480E994FF12
:10077E00401602079AC3E8947FE9940050030207DB
:10078E009A787F790002079A788079FF8849894A9A
:10079E0022E5492546F8E54A3547F9854A20E430F1
:1007AE000701F43548FA30E709C3EA94F040150220
:1007BE0007D8C3EA940F50030207D878FF79FF7A5F
:1007CE000F0207D8780079007AF0C3E524956150BE
:1007DE000AC374019524500B0207F6E54A20E70E72
:1007EE000207F6E54A30E706884689478A482278A6
:1007FE00A5E6FAC3E54933F8E54A33F91206B7E937
:10080E0030E70BC3E89480E994FF40130131C3E84D
:10081E00947FE9940050020131787F79000131789C
:10082E008079FFE820E715C3E52398F84009C3E86F
:10083E00940140030208587801020858E8F4240194
:10084E002523F8400302085878FF884B2278A6E645
:10085E00FAA847A9481206B7E930E70CC3E8940195
:0F086E00E994FF401602088DC3E894FFE9940057
:10087D00500302088D78FF790002088D780179FF09
:10088D00E920E715C3E54B98F84009C3E89401400A
:10089D00030208B478010208B4E8F42401254BF8EA
:1008AD0040030208B478FF88242278FFC2642069CF
:1008BD003D206A12D264C3E541940A4009C3E5257F
:1008CD0094405002C26479A1E76023E541601F7432
:1008DD00FF8541F0848539F0306A0375F005A4F881
:1008ED00C5F0600278FFC3E895645002A864886380
:1008FD0022C3E54094C8E5419400E56350031421FB
:10090D000F046002F563220209172275E890227820
:10091D0083E6FFE5E820ECF7A8BDA9BE0570C3E5A9
:10092D007094084052757000E9FA79A0E76044EAC6
:10093D007007E571601B020952C3E895716010E5FF
:10094D00715006600C1402095E0460F902095EE53F
:10095D0071F571C39472401B7561C0C3940440134B
:10096D00756180C39404400B756140C394044003CA
:10097D0075610075BB0922E5612410500274FFF505
:10098D00617982B7040221ABC3A861E524985002B6
:10099D00A824C3E895634002A86388258826E570DE
:1009AD00B4070375BB1022743279A787F0A4C5F084
:1009BD00A2F733F8C3E895614002A8618822882424
:1009CD00882588268864227540007541F022C2AFC3
:1009DD0075C820A8CCA9CDAA3A30CF010A75C82474
:1009ED00D2AFC3EA13FAE913F9E813F8AB3BAC3C09
:1009FD00883B893CC3E89BF8E99C20690A547FF940
:100A0D0030670241F54152AD3D8A3DF9EA9D547F73
:100A1D00FA600478FF79FFAE3EAF3F8B3E8C3FA866
:100A2D003BA93CC3E89EF8E99FF9C3E54113FBE5FB
:100A3D004013FAE82AF540E93BF54150067540FFB1
:100A4D007541FF419CAA40AB41AC40AD417E047F56
:100A5D0002C3EB940440021E1FC3EB940840021E18
:100A6D001FC3ED13FDEC13FCDEF7C3EA9CFAEB9DFF
:100A7D00FBEF6009C3E913F9E813F8DFF7EA28FA89
:100A8D00EB39FB8A408B4150067BFF8B408B41C37A
:100A9D00EB94025002D2673069047F0341C778920C
:100AAD00E6FFC3E537948240110FC3E53794A040AC
:100ABD00010FC3EF940640027F057E02E541C45449
:100ACD000FF9E541C454F0F8E540C4540F28F8C3BC
:100ADD00E89EFAE99400FB4009C3EA9402EB940006
:100AED0050047A02E4FB6141AA40AB41EBC4FEEA3B
:100AFD00C4540F4EFCC3EA9CFAEB9400FBC3E813FD
:100B0D00C313F8EA28FAEB3400FB8A408B41C3EBA0
:100B1D0094024002C2677802EBC4FE7B00EAC45423
:100B2D000F4EFAC3EA98FA4005C3940250027A02B6
:100B3D007892E6FF3060026141855192855293D2E1
:100B4D006043E680C3E49AF8E49BF9C3E833F8E91F
:100B5D0033F930670261D4E8FAE9FBD3E913FDE814
:100B6D0013FC88518952C3EF94036038EF20E00DD8
:100B7D00E82CF8E93DF9ECFAEDFB020B9DE828F8BD
:100B8D00E939F9C3E82402F8E93400F97AFE7BFF6C
:100B9D00C3EF9403400E8A538B54884D894E8C4F6E
:100BAD008D508108885389548A4D8B4E8C4F8D50B2
:100BBD003069127553F07554FF754FF07550FF7510
:100BCD0051F07552FF8108E8FAD3E813FC8851C340
:100BDD00EF94036020EF20E007E82CF8ECFA61F4C5
:100BED00E8282402F87AFEC3EF940340088A53885C
:100BFD004D8C4F810888538A4D8C4FE568C3335017
:100C0D0002646BF5683060028112753402D2604364
:100C1D00E680E52D5406602DA840A941C3E913F9DE
:100C2D00E813F8306904E92440F9C2AF53E67F7543
:100C3D009100C3E498F594E499F595759104D2600B
:100C4D0043E680D2AF22D265754300752000306C2B
:100C5D0003752040020C72D265754300752040303B
:0E0C6D006C0375200078017901206720E52DC9
:100C7B0054066002C2657914E541C313700104F890
:100C8B00C3941440027814306904781B791BC3E8B1
:100C9B0033F8C3E933F9206010E543600C30690386
:100CAB00D53404D26DA129911A0543E59B5440B567
:100CBB002002A11330690908C3E89940011881A1EA
:100CCB0020650A08C3E8994002817281A1C265C2FE
:100CDB00AF53E67F7591003067127594007595FCE4
:100CEB00759104D26043E680D2AF8172AE40AF41C2
:100CFB00C3EE33FEEF33FF50047EFF7FFFC3E49E52
:100D0B00F594E49FF59581EBC3E533940150028193
:100D1B00723065028172D802A12781A1C26DC2AF68
:100D2B0053E67F7591008553948554957591048591
:100D3B004D92854E93D26043E680D2AFE52D54069B
:100D4B006008206A020533020D65306D0D206C0AB8
:100D5B002065071581158102162322780030640562
:100D6B003065027801E53775F007A4F9E5F028F551
:100D7B00F0E9A2F013A2F113A2F213F537C39478A2
:100D8B005003753778C3E53795384008D266C29261
:100D9B00C294C296306002A19F854F92855093D228
:100DAB006043E68022D287207D16C2AF754202C215
:100DBB0095D293306202D296D2AF759F80020FAB61
:100DCB00C2AF754202C295D297306202D292D2AFB5
:100DDB00759F80020FABC287307243207D20C2AF5C
:100DEB00754203900165757B20C296C297306204F1
:100DFB00D294C101D295D2AF759F89020FABC2AF0E
:100E0B00754203900165757B20C292C293306204D8
:100E1B00D294C121D295D2AF759F81020FAB207DA9
:100E2B0017C2AF754203900140C296306202D29452
:100E3B00D2AF759F89020FABC2AF754203900140D1
:100E4B00C292306202D294D2AF759F81020FABD2A5
:100E5B0087207D16C2AF754204C293D297306202CF
:100E6B00D294D2AF759F81020FABC2AF754204C251
:100E7B0097D293306202D294D2AF759F89020FAB97
:100E8B00C287307243207D20C2AF7542059001545A
:100E9B00757B08C294C295306204D292C1ABD293D7
:100EAB00D2AF759F80020FABC2AF75420590017632
:100EBB00757B80C294C295306204D296C1CBD29717
:100ECB00D2AF759F80020FAB207D17C2AF75420565
:100EDB00900136C294306202D292D2AF759F8002DB
:100EEB000FABC2AF75420590014AC2943062EBD290
:100EFB0096D2AF759F80020FABD287207D16C2AF03
:100F0B00754206C297D295306202D292D2AF759FCC
:100F1B0089020FABC2AF754206C293D29530620203
:100F2B00D296D2AF759F81020FABC287307243202E
:100F3B007D20C2AF754201900176757B80C292C253
:100F4B0093306204D296E155D297D2AF759F81024E
:100F5B000FABC2AF754201900154757B08C296C2AC
:100F6B0097306204D292E175D293D2AF759F89020A
:100F7B000FAB207D17C2AF75420190014AC2923070
:100F8B006202D296D2AF759F81020FABC2AF754290
:100F9B0001900136C296306202D292D2AF759F8910
:100FAB00C26622900134757B00C292C294C296C273
:100FBB0093C295C297C26222788076090876090897
:100FCB0076040876FF0876030876FF08760908761C
:100FDB0003087601087601788C76010876FF08768F
:100FEB00FF0876FF0876FF0876FF0876030876FF82
:100FFB000876FF0876FF0876250876D0087628084D
:10100B0076500876040876FF087602087600087694
:10101B007A0876FF087601087601087600087603D1
:10102B00087600227887E6FFC272BF0302D272787D
:10103B0088E6C394036008C27DE630E102D27DC22C
:10104B007E7889E630E102D27EC3EF9402600875A8
:10105B008E01D273021067758E00C273227880E600
:0F106B00149000809378A5F67881E614900080A9
:10107A009378A6F67886E61490008D9378A7F6788A
:10108A0086E6F539C394025003753902789CE675F1
:10109A0038FFB402037538A0B4030375388278A305
:1010AA00E61490009A93F566120FAE22C2A4C2A06B
:1010BA00789DE6B40104D2A4C2A0B40204C2A4D2A8
:1010CA00A0227896E6FA7897E6FB7888E6B40305D4
:1010DA00C3EB940EFB307F047A007BFFC3EB9AFCD0
:1010EA00C3948250027C827572000572EC8572F09C
:1010FA00A4C3E5F0947D40F222D27F11CC120604FB
:10110A007A007B007C101205FAE55C2AFA74003B2F
:10111A00FBDCF37C04C3EB13FBEA13FADCF7FEC235
:10112A007F11CC22E5EF20E6037520000520903FD1
:10113A00FFE520146006901FFF146000930460030B
:10114A0075EF1253D9BF7581C043FF801205F5753B
:10115A00EF0243B203E5B3240220E70DF521E5E3EC
:10116A0020E0068521B343E301120FAE7580FF75B7
:10117A00A48075F1F075D4BF75900275A5FC75F25F
:10118A00FD75D50275A61175A0EE75F3F175E241EC
:10119A00120FAEE4F8F6D8FD756801120FC31216E5
:1011AA007C78988673753001C2AF12060E12061E3D
:1011BA0012060412062512060412062C120604C28E
:1011CA00AF78FA79FA308607D9FBD8F7021C0011F2
:1011DA002F116811B611CC78988673120FAE75A9C3
:1011EA000075B680757A0075881075890275C824ED
:1011FA0075910475D84075A82275B80275E6907580
:10120A009B80759D0075D10E75BCC075BB0975BAFA
:10121A001175E8801205F5D2AF120914753600531C
:10122A00DACF207E0343DA20307E0343DA1043DA32
:10123A0001C2D8C27112060ED2617B037A0CE55B39
:10124A0070077A0CDB030211C9120604207003022C
:10125A0011C9C270E55CC3940240E1E52F541F85B1
:10126A005E5DF55EB55DD5DAD5C26153DACF207E13
:10127A000343DA20307E0343DA10C2D8C27178A25F
:10128A00E67008D274E52F54E0F52FC2757529006F
:10129A00120609307409C3E529940A4002D275126C
:1012AA0005FA78023074027800C3E55C9840F0C20F
:1012BA00AF12061E12061E12061ED2AF12060E75B7
:1012CA004C007888E6B4030261A81205FA788CE625
:1012DA00C3940150030213A8E530C39401500302DA
:1012EA0013A8207435C3E55C94FF50030213A8C207
:1012FA00AF120633D2AF120609C3E55C940150EF70
:10130A00C2AF12061E1205FF12061ED2AF1206093E
:10131A00C3E55C94FF40E90218247F02D27F11CC16
:10132A00120609C2AFC27F11CCAE5CC3E55C947FE2
:10133A00D2AF40741205F5C2AF120633D2AFDFDC6A
:10134A003103C3EE7897F612060E1216BE1217A7CD
:10135A007F0AD27F11CC120609C2AFC27F11CCAE6E
:10136A005CC3E55C947FD2AF50E61205F5C2AF12BA
:10137A00061E1205FF12061ED2AFDFD63103EE2477
:10138A00037896F612060E1216BE1217D612060920
:10139A0011CCC3E55C94FF500241EC021824C3E56A
:1013AA005C954C4003855C4C12060978017988E704
:1013BA00B403027805C3E55C98400241CCC2AF127F
:1013CA000633120633120633D2AF12060E753000F8
:1013DA00E4F531F5320531E531F4703F0532789A9A
:1013EA00E67819146012783214600D787D1460085A
:1013FA0078FA146003753200C3E53298401D120F63
:10140A00AE1205F5153275310078998673C2AF129E
:10141A000633D2AF789886731206091205FFE52AB9
:10142A00700530740221C978012074027806C3E578
:10143A005C9840A17888E6C394036003120609E524
:10144A002A70030211C9C2AF120FAEE4F522F523C6
:10145A00F524F525F526F567D2AF7885E6C333F589
:0E146A0065E4F544F545F546F547F548F5709F
:10147800F52CF52DF53775700875BB101205F512AA
:101488000918E5E820ECFBA8BDA9BEE97001F888B9
:101498007112091C75700875BB10112FC2AF7561E8
:1014A800FF1209B4852261852262852263D2AF7555
:1014B8002201752401752501752601856069756A03
:1014C8000175B69075A903757A017888E6B40307A3
:1014D800C27D307602D27DD268D269753300120F90
:1014E80004120F351209D41209DB1209D41209DBD0
:1014F8001209D4120C6412070E120D66120DB012E6
:1015080009DB120C53306E0312076A2067031208B6
:10151800B73067031208FE120D66120DE11209DBDF
:10152800120C64306E0312079F120D66120E5A12C7
:1015380009DB120C53306E031207FD120D66120EF2
:101548008B1209DB120C64306E0312085B120D66F5
:10155800120F041209DB120918120C53120D66122D
:101568000F3512091C1209DB306932856461856404
:1015780062856069756A0179187A0CC3E533994008
:101588000FC269D26A8A358564618564630215A5CC
:10159800C3E55C940140030214FB02162B306A1D5C
:1015A800206C1AE535147006C26AD26B81FBF535DA
:1015B800C3E55C940140030214FB02162B75360048
:1015C80078FA79A4E760027803C3E55F985054304D
:1015D8007404E52A604D7888E6B40317207D052059
:1015E8007607A1FB307602A1FB206C07D26C8564DC
:1015F80061A13A78F0306C058564617820C3E541D3
:1016080098500281FB306C1BC26CC27D307602D2CE
:101618007DD26A75351285646181FB0536E55C60AB
:1016280002C12E753600C2AF120FAE7887E6FE767D
:1016380002112F7887EEF6E4F522F523F524F52537
:10164800F526F565752C00752D0075A90075B68011
:10165800757A00D2AF120609120FAE78A4E66006BA
:10166800D292D294D296307409C3E53694044002DB
:1016780021C961DA901A0D7820121700E520B455B7
:101688000CA3121700E520B4AA0302169E120FC37A
:101698001216BE0216BD901A0378807B0A12170034
:1016A800A308DBF9901A0F788C7B19121700A3088E
:1016B800DBF9901A2822C2AF12173F121719901A95
:1016C80000740E121705A37406121705A3741512D9
:1016D8001705901A0378807B0A121704A308DBF910
:1016E800901A0F788C7B19121704A308DBF91217CC
:1016F80052121730901A2822E493F622E6438F01FB
:10170800538FFD75EF0275B7A575B7F1F0538FFECE
:1017180022438F02438F0175EF0275B7A575B7F1A4
:10172800901A0DF0538FFC22901A0D7455F1059004
:101738001A0E74AAF105227A3079D07820901A40CE
:10174800F100E520F709A3DAF7227A3079D0901A68
:1017580040E7F10509A3DAF922AB74A875BB0102C9
:101768007980BB02027981BB03027982BB040279CA
:1017780084BB05027986BB06027992BB070279878A
:10178800BB080279A3BB0902799CBB0A027988BB12
:101798000B027989E8F7227C0512060EDCFB22C2CF
:1017A800AF12061E12062512062C1206331205FF6A
:1017B80012061E12062512062C1206331205FF12F7
:1017C800061E12062512062C120633D2AF22C2AF0D
:1017D80012063312062C12062512061E1205FF12D7
:1017E800063312062C12062512061E1205FF1206D3
:1017F8003312062C12062512061ED2AF22AE74AF83
:1018080075C2AF12061E12061E12061E1205FFDE54
:10181800F21206331205FFDFF8D2AF221217A71211
:10182800179F12179F75740175750175760011055C
:101838007C05AD5C12060EC3ED955C70F5C3E55CE6
:101848009401400AC3E55C94FF40370218671217F9
:10185800611216BE1217A7C2AF75EF1212179FDCDE
:0F186800D10576C3E5769403500280C212179F14
:101877000575E5741490009F93F808C3E5759850B3
:101887000280A912179F12179F0574C3E574940C61
:1018970050028095120FC31216BEC2AF75EF121217
:0218A700179F89
:0319FD0002112EA6
:101A00000E0615090904FF03FF0903010155AA0188
:101A1000FFFFFFFFFF03FFFFFF25D0285004FF0259
:091A2000007AFF0101000300FF40
:101A400023506C6174696E756D3530417633232097
:101A500023424C48454C492346333930232020202B
:101A60002020202020202020202020202020202076
:101C0000C2AFC2D353D9BF7581C043B20343FF8073
:101C1000752438752503B1C975EF0275E24043F1AB
:101C20004053A4BF75D4FFD2867DFA780379E67C51
:101C300010752200752300901DD67B0675249875BB
:101C400025013086028142208608D8FBD9F9DCF7CD
:101C500081B4308608D8FBD9F9DCF781B4B189E4C6
:101C600093A3C39A6004DDC381B4DBDBB17B600264
:101C7000812B7B08E493FAA3B15CDBF87A30B15C8A
:101C8000752200752300B17BEAFCEBFDC3ED94FEE9
:101C9000400EB17B8A278B28ED30E0048A828B834B
:101CA000B17B7AC270D8C3ED94FE601350CEBD00F4
:101CB00025EC60097520007521FF0200008100A855
:101CC00027A9280809D804D90281D3B17FEA89AAB3
:101CD000F281C50D81A0C3ED94035049EDA2E092BD
:101CE000007AC5C3E5829400E583941C50902000DF
:101CF00010438F02438F0175B7A575B7F1F030001F
:101D00001FA827A9280809438F01538FFDD804D99C
:101D100002A12089AAE275B7A575B7F1F0A3A10DBC
:101D2000538FFC817C7AC1BD030CE493A3FAB140CC
:101D3000DCF8B138817C817EAA22AB23B15CEBFA5E
:101D4000EA6222752608C3E52313F523E52213F57D
:101D50002250066323A0632201D526EAB1C9B1C986
:101D600075260AEAF4200102D286300102C286B149
:101D7000C9C3134002C201D526EB22B17FEAFB2082
:101D80008602A17F308602A184752608AE24AF2585
:101D9000C3EF13FFEE13FEB1CDB1C9C3EA13308612
:101DA000024480FA30E703632201C3E52313F523DD
:101DB000E52213F52250066323A0632201D526D91C
:101DC000E52265236523F52222AE24AF250E0FDE22
:101DD000FEDFFCD20122424C48656C693437316326
:041DE000F390060175
:00000001FF
